:020000020000FC
:100000009CCE1895189518954ACDCDC81895189579
:1000100018CC18951895189518951895E3C5189546
:100020001895000000000000000E111B1115110EA4
:100030000E1F151F1F1B0E0A1B1F1F0E0E04040E82
:100040001F1F0E04000E04151F150404040E0E1FBE
:100050001F040E0000040E0400001F1F1B111B1FB5
:100060001F00040A110A04001F1B1111111B1F039A
:1000700003040E11110E0E11110E040E04060505D7
:10008000040418180C0A0909091B1B00040E1B0E96
:100090000400080C0E0F0E0C0802060E1E0E0602BF
:1000A000040E0404040E040A0A0A0A0A000A1F1DA8
:1000B0001D050505050F100E110E011E0000001F85
:1000C0001F0000040E040E04000E040E04040404B9
:1000D0000404040404040E040000021F02000000D3
:1000E00000081F0800000000101010101F00000A78
:1000F0001F0A00000000040E1F00000000001F0E79
:1001000004000000000000000004040404040004D3
:100110000A0A0A000000000A0A1F0A1F0A0A040F3E
:10012000140E051E041819020408130308141409F8
:1001300015120D060204000000000204080808045D
:10014000020804020202040804150E040E1504003D
:1001500004041F0404000000000006020400000064
:100160001F00000000000000000606000102040855
:1001700010000E11111111110E040C040404040ED0
:100180000E11010204081F1F02040201110E0206D3
:100190000A121F02021F101E0101110E0E11101E65
:1001A00011110E1F0102020404040E11110E11118F
:1001B0000E0E11110F01110E000C0C000C0C0000A2
:1001C0000C0C000C04080204081008040200001FB4
:1001D000001F0000080402010204080E11010204BD
:1001E00000040E11171517100E040A11111F11111A
:1001F0001E11111E11111E0E11101010110E1C12C5
:10020000111111121C1F10101E10101F1F10101E94
:100210001010100E11101711110F1111111F1111C3
:10022000110E04040404040E0F02020202120C1147
:100230001214181412111010101010101F111B1589
:1002400015151111111119151311110E111111118B
:10025000110E1E11111E1010100E11111115120D7C
:100260001E11111E1412110E11100E01110E1F0479
:1002700004040404041111111111110E11111111B2
:10028000110A041111111515150A11110A040A1188
:100290001111110A040404041F01020408101F0EA6
:1002A00008080808080E001008040201000E0202E7
:1002B0000202020E040A110000000000000000000B
:1002C000001F0C08040000000000000E010F110FB9
:1002D00010101E1111111E00000F1010100F01013F
:1002E0000F1111110F00000E111F100E0304041F37
:1002F00004040400000F110F010E10101619111143
:100300001104000C0404040E0200060202120C0088
:100310001012141814120C04040404040E00000A31
:10032000151511110000161911111100000E1111EF
:10033000110E00001E111E10100000070907010118
:1003400000000B0C08080800000E100E011E04042B
:100350001F040404030000111111130D00001111FA
:10036000110A040000111115150A0000110A040AEF
:1003700011000011110F010E00001F0204081F06DA
:10038000080810080806040404000404040C02020F
:100390000102020C1926000000000000000000000D
:1003A000000000000000000000000000000000004D
:1003B0001818000708080711040015000411150A91
:1003C000150A150A150000000000000000000000DA
:1003D0000000000000000000000006091C081C09C5
:1003E0000600000000000000000000000000000007
:1003F00000000000000000000000000000000000FD
:1004000000000000000000000000000000000000EC
:1004100000000000000000000000000000000000DC
:1004200000000000000000000000000000000000CC
:1004300000000000000000000000000000000000BC
:1004400000000000000000000000000000000000AC
:10045000001F0404111B1511000000000000000023
:10046000000000000000000000000000000000008C
:10047000000000000000000000000000000000007C
:10048000000000000000000000000000000000006C
:10049000000000000000000000000000000000005C
:1004A000000000000000000000000000000000004C
:1004B000000000000000000000000A1F101C1C10BB
:1004C0001F0E11151915110E0E11101C10110E0012
:1004D000000000000000000000000000000000001C
:1004E000000000000E111D1B1D1B0E0A001F04043E
:1004F000041F0000000000000004041F0404001F8B
:100500000E04040404040E04000C0404040E000091
:1005100000000000000000000000000000000000DB
:10052000000006000000000000000A000E111F106D
:100530000E1313121A16121200000E111C110E00C7
:1005400000000000000000000000000000000000AB
:1005500000000000000000000000000A000C04047D
:10056000040E0709111F1111111E10101E11111E6A
:100570001E11111E11111E1F111010101010060A4D
:100580000A0A0A1F111F10101E10101F1515150E34
:100590001515150E11010601110E11111113151962
:1005A0001115111113151911111214181412110724
:1005B000090909090911111B151111111111111145
:1005C0001F1111110E11111111110E1F1111111105
:1005D00011111E1111111E10100E11101010110EFC
:1005E0001F1504040404041111110F01110E0E153E
:1005F00015150E040411110A040A11111212121217
:10060000121F01111111110F0101151515151515E5
:100610001F15151515151F0118080E0909090E11CA
:1006200011191515151910101E1111111E0E110199
:100630000701110E1215151D1515120F11110F05B9
:10064000091100000E010F110F0F08040E11110EF9
:100650000C12141E11110E00001E12101010000EAC
:10066000010F11110E00000E111F100E00001515C4
:100670000E151500000E1106110E000011131519AC
:100680001100041113151911000011121C12110090
:100690000007090909190000111B151111000011AB
:1006A000111F111100000E1111110E00001F111168
:1006B000111100001E11111E1000000E1110110E5C
:1006C00000001F04040404000011110F011E0000AB
:1006D0000E15150E040000110A040A110000121272
:1006E000121F01000011110F010100001515151551
:1006F0001F00001515151F01000018080E090E0037
:10070000001119151519000010101E111E00000E01
:100710001107110E000012151D151200000F110F08
:1007200005192020202020202020202020202020EB
:1007300020202020202020202020202020202020B9
:100740002020202122232425262728292A2B2C2D4E
:100750002E2F4F3132333435363738393A3B3C3D22
:100760003E3F404142434445464748494A4B4C4D31
:100770004E4F505152535455565758595A5B2F5D4E
:100780005E5F606162636465666768696A6B6C6D11
:100790006E6F707172737475767778797A28D12953
:1007A000E97F060704FFFF85868702898A8B8C8D87
:1007B0008E8F902727CBCA95969798019A9B9C9DE0
:1007C0009E9FA0A1A2A3A4A5A6A7A2A9AAABACADD7
:1007D000AEAFB003B2B3B4B5B6B7B54EBABBBCBDDD
:1007E000BEBF41A042A1E045A3A4A5A64BA74D488A
:1007F0004FA8504354A9AA58E1ABACE2ADAE05AF47
:10080000B0B161B2B3B4E365B6B7B8B9BABBBCBDF9
:100810006FBE7063BF79E478E5C0C1E6C2C3C4C5EA
:10082000C6C7868F98A1AA0000000000858E97A0F9
:10083000A90000000000838C959EA70B3331320085
:10084000848D969FA81B3937380F879099A2AB11DA
:100850000403011088919AA3AC141A090615808923
:10086000929BA413050C0712818A939CA50D363424
:100870003508828B949DA60002301900B3BCC5CE0A
:10088000D70000000000B2BBC4CDD60000000000BD
:10089000B0B9C2CBD40B33313200B1BAC3CCD51B03
:1008A0003937380FB4BDC6CFD81104030110B5BE17
:1008B000C7D0D9141A090615ADB6BFC8D113050C97
:1008C0000712AEB7C0C9D20D36343508AFB8C1CAA9
:1008D000D3000230190098A1C5CED7000000000057
:1008E00097A0C4CDD60000000000959EC2CBD40BCB
:1008F00033313200969FC3CCD51B3937380F99A2BC
:10090000C6CFD811040301109AA3C7D0D9141A096D
:100910000615929BBFC8D113050C0712939CC0C942
:10092000D20D36343508949DC1CAD3000230190067
:100930006770793A7B0000000000666F782D3D00FB
:1009400000000000646D765F400B33313200656E4D
:1009500077222A1B3937380F68717A3C7D110403DE
:10096000011069725B3E20141A090615616A73B1A1
:100970003F13050C0712626B745D2F0D363435087A
:10098000636C755EB900023019004750593B28006E
:1009900000000000464F582B260000000000444D88
:1009A000565F240B33313200454E5722251B393711
:1009B000380F48515A2C29110403011049525B2E5B
:1009C00020141A090615414A53822113050C0712F7
:1009D000424B545D220D36343508434C555E23009E
:1009E00002301900E6EFF83A7B0000000000E5EE67
:1009F000F72D3D0000000000E3ECF5FE400B333125
:100A00003200E4EDF6FF2A1B3937380FE7F0F93CE6
:100A10007D1104030110E8F1FA3E20141A090615AD
:100A2000E0E9F2FB3F13050C0712E1EAF3FC2F0D9E
:100A300036343508E2EBF4FDB90002301900C6CFB8
:100A4000D83B280000000000C5CED72B26000000B0
:100A50000000C3CCD5DE240B33313200C4CDD6DF49
:100A6000251B3937380FC7D0D92C291104030110A1
:100A7000C8D1DA2E20141A090615C0C9D2DB2113F9
:100A8000050C0712C1CAD3DC220D36343508C2CB9F
:100A9000D4DD2300023019008813A00FAC0DB80B71
:100AA000C409D007DC05E803F401FA0020534854D8
:100AB0005249482D5052494E5420444953504C41BC
:100AC0005920534D3830372E33312020762E312E99
:100AD0003520525553204431534D3830372E333161
:100AE0002020762E312E35205255532044320B0BC8
:100AF0000B0B0B0B0B0B0A0A0A0A0A0A0A0A090952
:100B000009090909804020100804020180402010D2
:100B100008040201804020100804000000000000CA
:100B200000000101010101010101020202020202B1
:100B300001020408102040800102040810204080B7
:100B40000102040810207201EC0000000091EC008A
:100B500008950FEF0ABB04E10BBB00E407BB0FE0F5
:100B600008BB01E004BB0FEF05BB01BB02BB07E004
:100B700006B907B99F9905C001E00093EC005CD766
:100B800009C008E101BD05E001BD02E00093EC00F1
:100B9000AAD1CDD203D000D67894089500E002BB4C
:100BA000A89874D101E0068B00EC14ED21E030E050
:100BB000008311832283338332BF0DE701BF0BE033
:100BC00003BF09B7016009BF3687089530E02223CB
:100BD00039F000FD05C01695079533953217C8F317
:100BE000032F0895BA93AA938A93FA93EA933A92B9
:100BF0002A921A920A927A936A935A934A933A9350
:100C00002A931A930A938FB7ADEEB0E00D911D9120
:100C10002D913C911397012B022B032B49F00D9141
:100C200012960ED1204030403C932E931E930E938B
:100C3000FD0104811581012B39F0048101D1048368
:100C40001583012B09F4D3D5FD0106811781012BF2
:100C500041F00681F5D006831783012B11F400E0E3
:100C6000048B00851185012B59F408EE13E00087F1
:100C7000118701E0168510271687012F14D204C0B2
:100C80000085DED000871187FD0102851385012BC9
:100C900021F00285D5D00287138707850023A9F0AC
:100CA0000489002391F400E007870589033019F4D3
:100CB000C2D00CE109C0043019F4BDD00DE104C06C
:100CC000023019F4B8D00EE1048B0089005049F0CD
:100CD0000A9561F10A9509F442C00A9509F475C0B4
:100CE00027C0B1D00689A1F4002309F087C09799E5
:100CF00004C00FEF02BBA89881C0A89904C00EEFF2
:100D000002BBA89A7BC002B3000F016002BB76C091
:100D1000002331F00EEF02BBA89A00E0068B6EC0F4
:100D200000890395008B0AE0018B68C08CD019F410
:100D300000E0008B63C07AD009F060C02AE046B3BF
:100D40004F7088D0042B6DD0028B29E002B310E0E5
:100D5000A89911E066D0038B00890395EACF6BD088
:100D6000238930E00AE0029F22894091790146FD03
:100D70000DC043FF08C047FF03C0E6EDF8E017C011
:100D8000ECE7F8E014C0E2E2F8E011C045FD08C06D
:100D900043FF03C0EEE3FAE00AC0E4EEF9E007C067
:100DA00043FF03C0EAE8F9E002C0E0E3F9E0E00D48
:100DB000F11DE20FF31F0491FD01048B0489058BE3
:100DC000348735870AEF018BC7CF3DD079F42ED019
:100DD000A9F400E0008B048515850D3D154010F049
:100DE00001E0078701E0068B00E084CF0AEF018B6A
:100DF000048515850F5F1F4F048715878FBF0991E5
:100E00001991299139914991599169917991099053
:100E1000199029903990E991F9918991A991B99105
:100E2000189500951095D2DEFD01089501890A9567
:100E3000018B0023089500ED17E0068317830895C2
:100E400001501040089526B32F7004D0022B0F3F9D
:100E50001340089503B310E00E77000F000F111F29
:100E6000000F111F089504EF11E010D004831583C3
:100E7000089500E00BD004830583089507D000E0B7
:100E800006830783048B08952FB7F894EDEEF0E006
:100E90000895FADF02851385012B11F001E001C0EE
:100EA00000E02FBF0895F0DF028713872FBF08955A
:100EB000399803C039980EC0399A0FD0000000004D
:100EC00000000000389800D00AEC0A95F1F700C045
:100ED0000895399A02D0389808953A98389A0BBBF9
:100EE000000000000895A9D001E09BD001D0E4CF1C
:100EF00006E097D00CE095D008E483D009E48DD0CB
:100F00000AE48BD00BE486D00CE4D2DF0BE1D4DF13
:100F10000DE4CEDF05E1D0DF0EE47CD00FE48AD013
:100F200000E575D001E570D002E568D003E563D037
:100F300004E564D005E568D006E569D007E57AD018
:100F400008E56BD009E569D00AE55BD00BE565D013
:100F50000CE563D00DE56ED00EE553D00FE56AD0F9
:100F600000E646D001E644D002E651D003E64CD07C
:100F700004E641D005E648D006E649D007E65AD057
:100F800008E633D009E631D00AE62CD00BE642D091
:100F90000CE640D00DE63ED00EE624D00FE64AD057
:100FA00000E748D001E746D002E744D003E742D04B
:100FB00004E740D005E73ED006E73CD007E73AD04B
:100FC00008E738D009E736D00AE734D00BE732D04B
:100FD0000CE730D00DE72ED00EE72CD00FE768DFFE
:100FE00000E0089565DF0EE167CF62DF00E164CFC6
:100FF0005FDF08E161CF5CDF08E05ECF59DF0CE125
:101000005BCF56DF0FE158CF53DF09E055CF50DFFC
:1010100006E052CF4DDF01E14FCF4ADF04E04CCF75
:1010200008E346DF0FE11EE401501040E9F700C07D
:10103000000008953DDF00E03FCF0FEF19EF000003
:1010400001501040E1F700C000C0EADF08E330DFE4
:1010500007E512E001501040E9F700C0000008E386
:1010600027DF0FE113E001501040E9F700C0000056
:10107000D7DF08E0D6CFAD01E0E3F1E024892160BD
:10108000248BDF0107C0AD0166D024892260248B48
:10109000A7E3B1E027E0F80131918F013D932A9554
:1010A000D1F7DA010895009343010895BA93AA9302
:1010B0009A93382E2FB6F894B801842FA0E3B1E0AC
:1010C000FD010589002311F000E02BC004E011E0D0
:1010D0009CE242E257E0FB010190BF011124400D68
:1010E000511DFA014491F80141938F019A9589F7B6
:1010F0008D01025F1F4F43E0F90151919F01F801FB
:1011000051938F014A95C1F7882311F08D3218F061
:10111000FD01118A05C001E0FD01018B8A95828BDA
:1011200001E02FBE832D9991A991B9910895B1D174
:1011300008EC19BD08BD1FBD03E00EBD00C009B716
:10114000006209BF089507D0008D002319F000E068
:10115000008FF5DF0895E0E3F1E008952497402F34
:10116000FADF068508830785098300890A830881D9
:1011700019812A813B8155E0459F402DEBD5202FD9
:101180002F7100E024FB0EF401E023FB0EF402605B
:1011900022FB0EF4046021FB0EF4086020FB0EF429
:1011A000006124960895BA93AA938A93FA93EA93D6
:1011B0003A922A921A920A927A936A935A934A938B
:1011C0003A932A931A930A938FB763D1A0E3B1E0BD
:1011D000FD010189002351F00389002339F00FE557
:1011E000228930E0F901EC5FFE4F0083FD010789A1
:1011F00024E031E0200F311F16891050A1F01A951C
:1012000049F11A95C9F11A9509F442C01A9509F4E1
:1012100084C01A9509F495C01A9509F4D9C01A9595
:1012200009F413C120C111E0158B002319F400E863
:1012300041DE05C021503040F90100814ADE36D13F
:1012400008F414C100E0078B06890395068B00E0C3
:10125000058B0CC111E0158B002319F400EC2ADE7C
:1012600003C0F901058935DE21D108F4FFC00AE386
:1012700030DE00E0FD01E7CF002319F406E91ADEB5
:1012800002C000E026DE0DD1023008F4EFC0DACF54
:10129000002319F400E40EDE3EC0013031F401E019
:1012A000058B00E05BDF15DE36C0023011F401E48F
:1012B000F2CF033011F401E0F5CF043011F402E471
:1012C000EACF053011F402E0EDCF063011F403E46B
:1012D000E2CF073011F403E0E5CF083011F404E465
:1012E000DACF093011F404E0DDCF0A3021F400E058
:1012F000058B05E4D0CF0B3011F400E0D4CF0C30D7
:1013000011F406E4C8CF0D30C1F30E3011F407E438
:10131000C2CF0F3091F3C2D0B8CF048900FF07C00D
:101320000E7F048B06890395068B00E09EC001FFAB
:1013300005C00D7F048B06890E5FF6CF07E0068B94
:1013400095C0002319F400E7B5DD3CC0013011F46D
:101350000C9137C0023011F401E7F6CF033011F4DD
:1013600001812FC0043011F402E7EECF053011F4F3
:10137000028127C0063011F403E7E6CF073011F4ED
:1013800003811FC0083011F404E7DECF093011F4E7
:10139000048117C00A3011F405E7D6CF0B3011F4E1
:1013A00005810FC00C3011F406E7CECF0D3011F4DB
:1013B000068107C00E3011F407E7C6CF0F3011F4D5
:1013C00000E087DD6BD008F451C000E0078BB6CF9A
:1013D000002311F408E7B8CF013011F40781F1CFF1
:1013E000023011F409E7B0CF033011F40085E9CFE2
:1013F000043011F40AE7A8CF053011F40185E1CFDC
:10140000063011F40BE7A0CF073011F40285D9CFD5
:10141000083011F40CE798CF093011F40385D1CFCF
:101420000A3011F40DE790CF0B3011F40485C9CFC9
:101430000C3011F40EE788CF0D3011F40585C1CFC3
:101440000E3009F0BBCF0FE77FCF018D0395018FE1
:10145000053138F000E0018F01E0008F09B70F7D02
:1014600009BF00E06CCF00E0068B078B8FBF0991AE
:1014700019912991399149915991699179910990DD
:10148000199029903990E991F9918991A991B9918F
:10149000189500E010E00DBD0CBD089502D000319C
:1014A0000895FD0107890395078B0895FADF073139
:1014B0000895A89519D075D10FE91FE0015010408B
:1014C000E9F700C000000AE411E00BD13FDB023075
:1014D0004091760109D019F4E9DD35DE01C0BBD2B7
:1014E0008FD1002331F3FFCF27E731E00AE411E089
:1014F000089501E000937A01089501E000937C01D2
:1015000000E010E0D0CC00937D01089500938101AC
:101510000895009380010895BD01D901FA01248145
:10152000222361F41CD020E005C030E2FD0131939C
:10153000DF012395FA0136812317B8F32481213086
:1015400049F420E003C030E23D9323953681231710
:10155000D0F305D0FA0106810A5EDB01089526E189
:10156000F80131918F013D932A95D1F70895AC018F
:10157000F8013081E22FF0E03197E13020E0F2070E
:1015800044F0CF01F801218120830F5F1F4F0197A5
:10159000C9F7F8013083CA010895BD01AC01822F5B
:1015A00090E0020F191F01501040F80120810197AF
:1015B000813030E093074CF0DC01F8013291F80102
:1015C0003083015010401197C1F7F8012083CA0100
:1015D000DB0108959A938A93C80180D0013011F0FD
:1015E000002341F44AE751E022E831E08C0194DF26
:1015F0000093DA0173D0023011F0002349F44AE776
:1016000051E02EEA31E046968C0186DF0093DB0143
:10161000899199910895EAE7F1E01381012F0F7004
:1016200039F000E00483012F017149F000E00FC0A0
:10163000012F007F11F001E0F5CF00E00895012FA8
:10164000027211F001E003C01474B9F302E00583E3
:101650000681073190F707810A3078F701E0089595
:101660006ED0D80116DC002391F5CD0137D00130C2
:1016700011F0002371F42091DA0100917E01002322
:1016800002E811E011F473DF01C087DFE2E8F1E066
:101690001FD024D0023011F0002381F42091DB010F
:1016A00000917E0100230EEA11E011F460DF01C019
:1016B00074DFDC015696EEEAF1E00AD0E8E9FAE0E0
:1016C0000091810112E0019FE00DF11D35D03CC079
:1016D00006E111911D930A95E1F7089500917F01AC
:1016E00008952DD0C801AAE7B1E0FD0102810023D1
:1016F00029F000E002830C9301831DC00C910023AC
:10170000A9F000E00C9387DF0023A9F08C0162DFD1
:1017100008E91AE0FD01278132E0239F000D111D29
:10172000F8010AD001E0FD01018303C0018100231B
:1017300011F08C0195DF08C005911491B4CBBA93D8
:10174000AA939A938A93089589919991A991B991AD
:101750000895BA93AA939A938A938CEA9AE0AAE49A
:10176000B1E00FD082EC9AE0F1D9023011F488EDAB
:101770009AE0A0E6B1E005D089919991A991B9913B
:10178000089506E1FC011591CF011D930A95D1F74B
:101790000895DFD9DEDF8DCE0FEF0FB900EC0DB964
:1017A00008951B2E2A2E0FB6F894A801ECEDF1E057
:1017B00003810023C1F004E112E06CE2D8017D91C5
:1017C0008D01DA017D93AD016A95C1F700E412E065
:1017D00043E0D8015D918D01D9015D939D014A954A
:1017E000C1F700E003830FBEA22DB12D0895ECEDEB
:1017F000F1E000E0008302833CDB0FEF0FB90895B6
:101800001FB7F894ECEDF1E000810023B9F40481F6
:10181000B69907C0002329F401E0048303E005839F
:101820000DC0002359F0B69B03C000E0048307C03D
:1018300005810A95058311F401E0F8CF00E01FBF90
:1018400008954A92BA93AA939A938A93FA93EA9341
:101850003A922A921A920A927A936A935A934A93E4
:101860003A932A931A930A934FB60EB12FB106708A
:10187000B1F0BDDF4FBE099119912991399149917C
:101880005991699179910990199029903990E9912C
:10189000F99189919991A991B99149901895A2EEE0
:1018A000B1E08CED91E0FC01428150E08D01040F2C
:1018B000151F3081332339F03A95D9F03A95C1F1AB
:1018C0003A9531F1D6CF2B3121F401E000830FE2BC
:1018D0000AC02D3121F403E0008308E004C02C315C
:1018E00041F602E000830183009101010FB9BBDAE8
:1018F000C1CF93D0E1F704E112E09D014FE2F9017D
:1019000051919F0185D0D9F701E0FC010383B1CF4C
:1019100084D069F70C91002319F00A9529F0A9CF1A
:1019200011968D01A8DBA5CF11968D01ACDBA1CF5F
:1019300077D0013029F40C910031C9F607D90FB9DD
:10194000FC010181002399F6FD0101811C911E5DBE
:1019500009F448C01B5009F44AC0115259F01A95B5
:1019600089F11A95B1F11A95B1F1125041F11A9518
:10197000A1F17FCF002339F4E4E1F2E00CE244D09E
:1019800009F477CFFCCF013039F4E4E1F2E006E16D
:101990003BD009F46ECFFCCF023039F4EAE2F2E03A
:1019A00006E132D009F465CFFCCF033009F061CFF6
:1019B000E0E4F2E003E028D009F45BCFFCCF009331
:1019C000760157CF002311F498DD53CF9CDD91DDD4
:1019D00050CF9FDD4ECF9ADD4CCF002309F049CF89
:1019E0004DDA47CF0CD009B70F7B09BF42CF07D0E4
:1019F000F89405B7006205BF889578943ACFA6D8C9
:101A0000013009F4D898089510E211930A950895C9
:101A1000F80151938F014A95089502D0002308954B
:101A200031813A953183F8012083FC0102810395CD
:101A300002835FB90181089500E010E00DBD0CBD87
:101A400004EB1BBD0ABD1FBD0BE00EBD09B7006452
:101A500009BFD89A08955B2F6A2FD801E4E0F1E01E
:101A60000CE21D9111930A95E1F7AEE3B1E003E0BA
:101A7000F90111919F011D930A95D1F7442311F0AB
:101A80004D3220F000E00093410106C001E00093D8
:101A900041014A9540934201A62FB52F0895BA936C
:101AA000AA939A938A93FA93EA933A922A921A9271
:101AB0000A927A936A935A934A933A932A931A937F
:101AC0000A933FB6DC9AA3E4B2E020E00EEE1AE0FF
:101AD000FD01428D50E0040F121FF801049110E047
:101AE000FD01E00FF21F2687DB9AFD01028D0395B1
:101AF000028F063108F0228F228D30E0E4E0FBE017
:101B000002D14491EEEEFAE0FED00491FD01E00F27
:101B1000F51F4687EAE1FBE0F6D00491F801E25CAC
:101B2000FE4F0081E0E3FBE0EED01491102311F0B2
:101B300011E001C010E0DB980000DC98FD01028D8F
:101B4000802F90E044E051E0400F531FFA01608184
:101B5000603831F420E331E0D9D0E4D0A9F0FDCFF2
:101B6000613831F427E331E0D1D0DCD069F0FDCF2A
:101B700022E230E0262E67E0629D200D311DC6D0A6
:101B8000F9011590D1D0E1F7FA016689603831F496
:101B900020E331E0B3D0BED0A1F0FDCF613831F405
:101BA00027E331E0ABD0B6D061F0FDCF22E230E0E8
:101BB00047E0469F200D311DA1D0F9017591ACD0B1
:101BC000E1F7209141012223F1F0209143012223EA
:101BD000D1F020E030E040914201401709F49D012E
:101BE00050E046964817590719F49D01295F3F4F69
:101BF000022F032B41F006E0F90151939F010A9552
:101C0000D9F70FE10083FD0121810C916FD0368B54
:101C1000038130E4239F328162D0258B0295007FBF
:101C200024812695202B248B0681248120FB20E013
:101C300027F93581330F330F322B202F2695269528
:101C40002695232B238B0295007F000F2781202BC5
:101C5000228B218500854AD0318B038530E4239F78
:101C600032853DD0208B0295007F24852695202B40
:101C70002787048500FB00E007F92585220F220F46
:101C8000202B2687112319F0022F016006871E964C
:101C90009D010CE0F90141919F0118E0DA9840FBA9
:101CA00016F4D99A01C0D998DA9A46951A95B1F7DF
:101CB0000A95002379F73FBE09911991299139912D
:101CC0004991599169917991099019902990399088
:101CD000E991F99189919991A991B9911895330F49
:101CE0003029202F22952F70232B0895000F000FED
:101CF000000F322F36953695302B0895AD01495F90
:101D00005F4F67E00895E20FF51F0895BD01E7E01A
:101D10000E2E0895F90171919F01FA017193AF019F
:101D20006A950895F90111909F01FB011192BF017D
:101D30000A94089500008895FECF0BEE0DBF00E0D9
:101D40000EBFC0EAD0E00ED0002309F01BD021DD89
:101D5000F1DFF0CF4A952AF036952795179507952C
:101D6000F9CF089501E0089520E006D0E9F708953D
:101D7000259102D0E9F708952D9301501040202FAE
:101D8000212B089586E49BE0FC0105911491FC0150
:101D90003296A591B491FC01349625913491422F4D
:101DA000432B19F0F901E4DF01C0DEDF06961BE0EA
:081DB0008C34910748F30895FB
:0400000300000000F9
:00000001FF
